:1000000000308A00C02900008A1D0A128A190A16C7
:100010008A11831A0F28A500030EA6001428831244
:10002000A500030EA600A6140A08AD00A50E04083C
:10003000A7002008A8002108A9002208AA00230878
:10004000AB002408AC0083128C308400801E2A2868
:100050008C1A4228270884002808A0002908A1003B
:100060002A08A2002B08A3002C08A4002D088A004F
:100070000A1A8A150A12260E83008312250EA61864
:10008000831609008A1174280A108A100A1182073F
:100090002034443449344F342534633420344434D8
:1000A000503400344D1B59284D080F39A1006028E9
:1000B00060284D080F39A00009302007A1006028F2
:1000C000003480304C02031C6628732820304C0218
:1000D000031C6E2880304C078400712860304C0768
:1000E00084004D08800000348C1E1F2964001A080B
:1000F000CA00351C952821304A0203198328233071
:100100004A02031D94288710B6012F08AE0035114E
:10011000351023304A02031D91280330CB00B5145B
:1001200094280130CB00B5101E2938083702031D72
:100130009C283515071011290D304A020319A428EF
:100140000A304A02031DD62805304B073602031930
:10015000AB280318AD283515D328B51CC2283A089A
:10016000CD0052202108CC00CC0EF030CC053B084D
:10017000CD0052204C082104AE07AE080319C22856
:10018000351507103519D3283708CC000D30CD00B0
:1001900061203708B9007F303702031DD128B7012D
:1001A000D228B70A071435148714112902303602F1
:1001B0000318E228B51CE2283A30360784004A08C2
:1001C0008000F72836084B020319E8280318F7289F
:1001D00004304B0736020318F7284B083602A000FC
:1001E0003130200784004A080002031D3515B51C74
:1001F000FF2808303602031CFF284A08AE073519CD
:10020000102905304B073602031C10293708CC0093
:100210004A08CD006120B70A803037020318B701C1
:10022000B60A351D1E297F303902031D1929B70171
:100230001C2901303907B7003514871474288A1136
:100240002A2820304702031C2929803047078400D0
:100250002C296030470784000008A10000343908C9
:100260003802031942290D30300203194229B80A15
:1002700080303802031C3D29B8013808C70021210D
:100280002108B0003008A10000340A3047020318EA
:100290004E2947083038A100532953290930470215
:1002A0004038A10053290034473084000008031966
:1002B0006A290130A100BF30A0006400A00B5D29B5
:1002C000A10B5B293030A000A00B64290000640062
:1002D000800B5929003487160C1E6C294908990097
:1002E000871683169818762983127129831287122C
:1002F0000034C71B8E290F30A000460EA0050A301F
:100300002002031886293030A00788294708A00753
:100310002008C80064004808C9006B210F30C605DA
:100320000A3046020318962930309829C713470827
:10033000C6074608C80064004808C9006B218A1136
:10034000B52A6400051EB2298101051EB229640088
:100350000108A000C4302002031CB1290030A10014
:10036000BE29A52946088600000085110730A00097
:10037000A00BB829000085150130A1008A11042CBA
:100380003F30A0002130840000308000840AA00BA0
:10039000C529A00184011F3083058712053083160B
:1003A00099002230980090308312980081308400A8
:1003B0008013FF3066000730A000A01DE72907303A
:1003C0008101813084000008C0390F38800064004A
:1003D000813084000008C03920048000D7306500D7
:1003E0008515FF30BD009830670007148714071586
:1003F0004430B1004930B2004F30B3000508FF3A35
:100400000739A00030302007B4009F30AF00340817
:10041000AF073514B701FF30B800FF30B900060848
:10042000C100C2010B138B138B1B132A8C30840069
:100430008016C0308B0439083802031D2A2A640054
:10044000981C262A071018120000181606084106E4
:10045000C2041B2A6400380A031D302AB801362A58
:10046000B80A80303802031C362AB8013808C700A1
:1004700021212108BE00B0012F2120302102031DBF
:10048000422A2F213E08A000513020020319552A8C
:10049000523020020319152B533020020319252B4B
:1004A0005430200203198A2B0F2C06084106C2047F
:1004B00041084206BC000608C100C2012F212F21BD
:1004C0002E302102031D872A43102F212108C0004E
:1004D0004008BF00383040020318722A3030400212
:1004E0000318732A102C30304002031C7E2A03109C
:1004F000BC0CBE010318BE0AC003732A0130BE053E
:1005000030303E07C4002E303F07C500992A4314FF
:100510003C08C600C60E0F30C6054608C700452178
:100520002108C4003C080F39C600C7004521210836
:10053000C500B51CA42A7130BE0034084407450725
:10054000BE07FF30BE06BE0A18123230C700542163
:100550002430C80064004808C9006B21B51CB52AC6
:100560003E08C6003730C7007929C6014608442036
:10057000C60AC80064004808C9006B21043046025E
:10058000031DB62A3408C80064004808C9006B215E
:100590002030C80064004808C9006B214430C800FE
:1005A00064004808C9006B215030C8006400480846
:1005B000C9006B214318FB2A2E30C800640048088C
:1005C000C9006B213F08C80064004808C9006B21BE
:1005D0003D30C80064004808C9006B214408C800C9
:1005E00064004808C9006B210A30C800640048084C
:1005F000C9006B21132B3D30C80064004808C900B6
:100600006B214408C80064004808C9006B214508F4
:10061000C80064004808C9006B210A30C8006400A3
:100620004808C9006B211816102C0B138B138B1B59
:10063000162B0710871007110830C600FA30C700C4
:100640005421C60B1E2B232B102C07112F212F21D9
:100650003D302102031D502B2F212108C600CD0063
:100660000B088B13A500522025088B042108C60017
:10067000C60EF030C6052F212108C700CD000B089B
:100680008B13A500522025088B0446082107BD00C6
:100690003D0866003D0886003D08C100C201812B6F
:1006A0000130C0002F212108BE0038303E0203185F
:1006B0005D2B30303E0203185E2B102C0F30BE0530
:1006C000BE080319672B0310C00DBE03602B400842
:1006D000FF3AC2052F212F2130302102031D7B2B31
:1006E0004008FF3ABD054008FF3AC1053D088600B5
:1006F0003D086600812B4008BD044008C1043D0848
:100700006600000085114C30A000A00B852B000076
:100710008515102C07112F21003066002F212F2165
:100720002108BF000D303F0203190E2C64005C301D
:100730003F02031DFF2B2F212108A0006E30200255
:100740000319BF2B723020020319C22B783020020C
:100750000319C52B663020020319E22B65302002F5
:100760000319E52B743020020319E82B63302002B3
:100770000319EB2B5C3020020319F82BFB2B0D30F7
:10078000BE00FE2B0A30BE00FE2B2F212108C60022
:10079000CD000B088B13A500522025088B042108DF
:1007A000C600C60EF030C6052F212108C700CD00B7
:1007B0000B088B13A500522025088B044608210442
:1007C000BE00FE2B0C30BE00FE2B1B30BE00FE2BED
:1007D0000930BE00FE2B2F212108BE0060303E02F2
:1007E000031CF52B6030BE02F72B4030BE02FE2BFF
:1007F0005C30BE00FE2B2F212108BE00012C3F08DB
:10080000BE003E08C600A129A108031D0A2C0D3018
:10081000BF000D2C2F212108BF00922B102C102C73
:100820002F210D302102031D102C07151B2A172C18
:02083000630063
:02400E00C500EB
:00000001FF
